:020000040000FA
:100000005BEF00F0E834E8343C0B0109C212C00990
:10001000C216C050F80B0609C06E000E026E320EFA
:100020001BEC00F0C282C2B2FED7C450026EC350B5
:1000300058EF00F0026AFE0F016E0400E86A025AEF
:10004000D8A01200010600D000D0F7D745EC00F090
:1000500002D042EC00F004E00450026E0350016E46
:1000600001501200D89001360236FF0FFBE201501A
:1000700058EF00F0D89002320132FF0FFBE201503E
:1000800058EF00F0036E010E03D0036E040E00D093
:10009000096E0450025C02E10350015C040ED8B00A
:1000A000010ED8B4020E0914D8A4FF0E58EF00F0C8
:1000B000000104001200D7EF04F0120C010C000C38
:1000C000010C000C000C000C080CD80C040CE30C08
:1000D000000C000C000C010C020C000C010CE200E6
:1000E000E200090C020C220C000C010C010C040CA7
:1000F000800C320C090C040C000C000C010C030CDD
:10010000000C000C050C090C210C000C010C000C5F
:10011000010C220C2F0C000C070C050C810C030C9D
:10012000030C000C0A0C050C010C090C050CA10CAD
:10013000010C090C010CA10C000C090C300C090C71
:10014000310C150C000C260CFF0C000C750C080C67
:10015000950C020C810C020CC00C050C090C190C3E
:10016000010C290C060C150C000C250C010C750C4F
:10017000010C950C060C810C020C950C020C810CE8
:10018000030CC00C8C0C010CA40C010CC80C010C51
:10019000D40C010CFC0C010C3C0C020C5C0C020C91
:1001A000700C020CC80C010C880C020CB00C020C78
:1001B000F00C020C0C0C030C200C030CC801D40135
:1001C000FC013C025C027002060C030C090C040CDE
:1001D000040C080C140C030C4D0C000C690C000CE6
:1001E000630C000C720C000C6F0C000C630C000C08
:1001F000680C000C690C000C700C000C200C030C3B
:10020000500C000C490C000C430C000C200C000C92
:10021000550C000C530C000C420C000C200C000C74
:10022000470C000C410C000C4D0C000C450C000C54
:10023000500C000C410C000C440C000C100C030C76
:10024000560C000C310C000C2E0C000C310C000C68
:10025000300C000C460C000C530C000C0A0C030C68
:10026000430C000C660C000C670C000C310C000CED
:100270000C0C030C450C000C500C000C310C000C49
:10028000490C000C6E0C000C140C030C4D0C000CF3
:10029000690C000C630C000C720C000C6F0C000C51
:1002A000630C000C680C000C690C000C700C000C4A
:1002B000200C030C500C000C490C000C430C000CDF
:1002C000200C000C550C000C530C000C420C000CC4
:1002D000200C000C470C000C410C000C4D0C000CC9
:1002E000450C000C500C000C410C000C440C000C94
:1002F0000E0C030C560C000C310C000C2E0C000CD8
:10030000310C000C460C000C530C000C0A0C030CB6
:10031000430C000C660C000C670C000C310C000C3C
:100320000C0C030C450C000C500C000C310C000C98
:10033000490C000C6E0C000C04011E51600B0008EF
:100340003EE1050E1F6303D0040E1A6F36D0060E71
:100350001F6301D035D0080E1F6309D01B0E126F2A
:10036000040E136F010E186F196B1D9326D0090E22
:100370001F6301D06AD0000E1F6301D07ED0010E32
:100380001F6301D09FD0030E1F6301D09BD00A0EC4
:100390001F630BD01C0E126F040E136F2251122715
:1003A000010E186F196B1D9308D00B0E1F631200FE
:1003B00024EE1CF0225120C4DBFF010E176F120047
:1003C000800E1E631200010E21630FD0BA0E126F51
:1003D000000E136F12C4F6FF13C4F7FFF86A08008B
:1003E000F5CF18F4196B1D83E8D7020E216312D0E4
:1003F000E20E126F000E136FE60EF66E000EF76E31
:10040000F86A0900F5CF18F409000900F5CF19F4CE
:100410001D83D3D7030E21631200F86AF76A2045C3
:10042000BC0FF66E010EF7220900F5CF12F408009A
:10043000F5CF13F412C4F6FF13C4F7FFF86A0800EF
:10044000F5CF18F4196B1D83B8D7010E176F2FEE77
:1004500071F00F0EDE6AE82EFDD724EE1CF0010EBF
:10046000DE6AE82EFDD720511B6F03E1050E1A6FDF
:100470001200060E1A6F09DA1200266B276B1E5146
:100480001F0B000803E11DB126830ED01E511F0B68
:10049000010801E109D01E511F0B020807E134D801
:1004A000DF50040B01E02681010E176F010E176368
:1004B0001200260E126F040E136F020E186F196BC6
:1004C0001D931200010E206309D01E511F0B00085E
:1004D00005E11D81030E1F631D916FD7000E206380
:1004E00012001E511F0B0208FBE122510F0BF8E016
:1004F0000BD8030E1F6303D0840EDF6E5ED7000E91
:1005000022AF880EDF6E59D724EE00F02245223547
:10051000E846E846D9261200000E6C6205D000516C
:100520003C0B340805E010D0040E6C62120015D0AC
:10053000000E166F000E176F186B196BFDDE000EA4
:10054000176379D046D977D0020E1663B0D057D84A
:10055000C80E00BD880E006F1200040E1A6306D08C
:1005600020516E6E050ED8B4030E1A6F010E16637D
:100570009ED005D8C80E04BD880E046F1200185115
:10058000106F1951116F000804E307E118510808B2
:1005900004E2080E106F000E116F1051056F185F06
:1005A0001151195B0451FC0B1111046F24EE26F05C
:1005B000115102E1105122E01DA312D012C4F6FF26
:1005C00013C4F7FFF86A0900F5CFDEFF0900100732
:1005D000FAE11107F8E2F6CF12F4F7CF13F41200A4
:1005E00012C4E1FF13C4E2FFE6CFDEFF1007FCE117
:1005F0001107FAE2E1CF12F4E2CF13F41200015135
:10060000106F18270051030B116F192314EE26F0F9
:1006100014C4D9FF15C4DAFF115102E110510AE0E8
:10062000E6CFDEFF1007FCE11107FAE2D9CF14F4A0
:10063000DACF15F412006D98000E17630AD0080E79
:10064000016F1E0E026F040E036F840E006F046FA5
:100650002CD01EAF1DD01951255D04E307E11851C0
:10066000245D04E224C418F425C419F488DF010EC3
:10067000166F080E016F1E0E026F040E036F800EC0
:10068000006F260E066F040E076FC80E046F0DD0A4
:10069000020E166F056BC80E046F080E016F260E52
:1006A000026F040E036FC80E006F6D981200000EEB
:1006B000166F080E016F1E0E026F040E036F880E78
:1006C000006F000E046F12000401140E6F6E000E16
:1006D0001A6F1D6B1B6BD9D8120004016DA60CD8C4
:1006E000010E1A6312006DBA1200686A696A6980A5
:1006F0006988020E1A6F12006D6A696A6D86010EB2
:100700001A6F120004016D6A696A000E1A6F1200F6
:100710000401000E1A5D23E068A402D069B424D855
:100720006DB2120068A002D069B039D868A802D0B2
:1007300069B816D868AC02D069BC28D868AA02D0BB
:1007400069BA26D868A202D069B227D8030E1A5D0A
:1007500006E368A604D069A602D0DEDE6896120021
:10076000698468986D8212006D9269946894120091
:1007700004011DA11200F8DF6D84100EDA6ED96A33
:10078000D92EFED7DA2EFCD76D941200689C120089
:1007900070B08DDF7090689A1200689212006A6AD9
:1007A000686A9F0E6B6E7B0E696E6E6A2FEE71F03B
:1007B0000F0EDE6AE82EFDD7160E706E68B66896CC
:1007C00068B6FDD76D9873DF1D911B6B030E1A6F12
:1007D000120004011E511F0B010802E1000E2263EA
:1007E0001200060E1F6327D0210E21630FD0060EC4
:1007F000126F010E136F12C4F6FF13C4F7FFF86AED
:100800000800F5CF18F4196B1D833CD0220E21632C
:1008100012D0260E126F010E136F140EF66E010E1B
:10082000F76EF86A0900F5CF18F409000800F5CF53
:1008300019F41D8327D01E51600B2008D1E1020E50
:100840001F6309D02E0E126F040E136F010E186F66
:10085000196B1D9317D00A0E1F6303D021C42EF409
:1008600011D0030E1F6309D02F0E126F040E136FE9
:10087000010E186F196B1D9305D00B0E1F6312002C
:1008800020C42FF4020E176F1200010EE96E14EE51
:1008900030F0080E1CD8010EE96E14EE39F0080E87
:1008A00000D0E66E2FEE70F0E950D9261A0EDF1256
:1008B000E944E846E84604EE04F0E926020EE1CFFA
:1008C000EBFF030EE2CFEBFF400EEF6E1200E66E81
:1008D0002FEE70F0E950D9261C0EDF12E944E846ED
:1008E000E84604EE00F0E926020EE1CFEBFF030E2E
:1008F000E2CFEBFFE550E92AE7CFEDFF880EEF6E80
:100900001200016E0401060E1A5D000ED89009E176
:10091000E944E846E84604EE04F0E926000ED890E3
:10092000EFBE1200020EEBCFD9FF030EEBCFDAFFC2
:10093000FF0EDB500160016EE92A0150ED6E04E00C
:10094000E6CFDEFFE82EFCD7400EEF16EF7C880ED8
:10095000EF120150D8801200016E0401060E1A5DDC
:10096000000ED89009E1E944E846E84604EE00F0BC
:10097000E926000ED890EFBE1200020EEBCFD9FF91
:10098000030EEBCFDAFFEC500160016EFF0EDB507F
:10099000ED6E015004E0DECFE6FFE82EFCD7400EFE
:1009A000EF16EF7C880EEF120150D8801200928073
:1009B00092820D0EC16EAE0EC06EF19E9380938238
:1009C0009384938681DE58EC00F0000E02EC00F078
:1009D0001C6E02C01DF0010E02EC00F01E6E02C083
:1009E0001FF01CC001F01DC002F0020E3DEC00F033
:1009F000136E02C014F013C001F014C002F0020E16
:100A000035EC00F01C6E02C01DF01EC001F01FC0CE
:100A100002F0020E3DEC00F0136E02C014F013C0A1
:100A200001F014C002F0020E35EC00F01E6E02C0A0
:100A30001FF0800E016E010E026E1DC004F01C50EE
:100A400026EC00F0136E02C014F07F0E016E020E51
:100A5000026E14C004F0135029EC00F0136E02C0B3
:100A600014F0800E135C1C6E010E14581D6E800E67
:100A7000016E010E026E1FC004F01E5026EC00F045
:100A8000136E02C014F07F0E016E020E026E14C0CF
:100A900004F0135029EC00F0136E02C014F0800E25
:100AA000135C1E6E010E14581F6E1EC020F01CC079
:100AB00021F00F0E8118136E000E146E0F0E13141A
:100AC000226E0BDE25DE58EC00F0010EE96E10EE12
:100AD00020F0030E16DF58EC00F0D8A076D775D7BB
:020000040030CA
:08000000E4FEFFF3FF7D9BFF0E
:00000001FF
